:020000040800F2
:1000000000040020E1010008490F00084D0F00081E
:10001000A10F00084D0F0008750F0008E30100084C
:10002000E3010008E3010008E3010008E5270008F8
:10003000E3010008E3010008E3010008E301000810
:10004000E3010008E3010008E3010008E301000800
:10005000E3010008E301000891390008BD390008F8
:10006000E9390008153A0008413A0008E3010008A0
:10007000E3010008E3010008E3010008E3010008D0
:10008000E3010008E3010008E3010008E3010008C0
:10009000E3010008E3010008E30100086D3A0008ED
:1000A000E3010008E3010008E3010008E3010008A0
:1000B000E3010008E3010008E3010008E301000890
:1000C000E3010008E3010008E3010008E301000880
:1000D000E3010008E3010008411100085511000880
:1000E000D53A0008E3010008E3010008E301000835
:1000F000E3010008E3010008E3010008E301000850
:10010000E3010008E3010008A1370008E30100084B
:10011000E3010008E3010008E3010008E30100082F
:10012000E3010008E3010008E3010008E30100081F
:10013000E3010008E3010008E3010008E30100080F
:10014000E3010008E3010008E3010008D12E0008E4
:10015000E3010008E3010008E3010008E3010008EF
:10016000E3010008E3010008E3010008E3010008DF
:10017000E3010008E3010008E3010008E3010008CF
:10018000E3010008E3010008E3010008E3010008BF
:10019000E3010008E3010008E3010008E3010008AF
:1001A000E3010008E3010008E3010008E30100089F
:1001B000E3010008E3010008E3010008E30100088F
:1001C000E3010008E3010008E3010008E30100087F
:1001D000E3010008E3010008E3010008E30100086F
:1001E00002E000F000F8FEE772B6394880F30888B4
:1001F000384880F3098838484EF60851CEF200019D
:10020000086040F20000CCF200004EF63471CEF2ED
:1002100000010860BFF34F8FBFF36F8F40F2000003
:10022000C0F2F0004EF68851CEF200010860BFF334
:100230004F8FBFF36F8F4FF00000E1EE100A4EF6C4
:100240003C71CEF200010860062080F31488BFF3F1
:100250006F8F02F005FB03F02BFA4FF055301F496A
:100260001B4A91423CBF41F8040BFAE71C49194A6A
:1002700091423CBF41F8040BFAE71A491A4A1B4B5A
:100280009A423EBF51F8040B42F8040BF8E70020F5
:100290001749184A91423CBF41F8040BFAE702F0B3
:1002A000E3FA03F06FFA144C144DAC4203DA54F83D
:1002B000041B8847F9E700F03FF8114C114DAC42A0
:1002C00003DA54F8041B8847F9E702F0CBBA0000C0
:1002D000000400200024002000000008000000208E
:1002E00000040020B03F0008002400202824002043
:1002F0002824002040390020E0010008E001000827
:10030000E0010008E00100082DE9F04F2DED108A12
:10031000C1F80CD0C3689D46BDEC108ABDE8F08FD3
:10032000002383F311882846A047002001F0D6FE61
:1003300001F086FE00DFFEE770B5204C0D2300259E
:1003400023706FF03F061F236570A570E57025715F
:100350006571A571E57125726672A372E57200F090
:10036000FFFC20B10F2325726672A372E57202F0C2
:100370000BFA044602F030FA0546D8B9104B9C42FD
:100380001AD001339C4218BF054641F2883404BF9D
:1003900001250024002002F001FA0DB100F0B6F8AA
:1003A00000F072FD00F01AFC204600F00DF900F09C
:1003B000ADF8F9E70024EDE70446EBE72824002038
:1003C000010007B008B500F087FBA0F120035842F8
:1003D000584108BD07B5054B02211B88ADF8043014
:1003E00001A800F0E5FB03B05DF804FBBC3B00088E
:1003F000064991F8243033B100230822086A81F8B5
:10040000243000F00DBC0120704700BF48240020BC
:100410002DE9F84F234C94F82430054688461746BA
:100420008BBB2E46DFF87C90002F38D094F824A0A8
:10043000BAF1000F05D12022FF214846266200F0C4
:1004400011FDCAF10805BD4228BF3D465FFA85FB94
:10045000AD0041462A4604EB8A0000F0D9FC94F82E
:100460002430A7EB0B079B445FFA8BFBBBF1080F13
:100470002E44A844FFB284F824B0D5D1FFF7B8FFCA
:100480000028D1D108E0266A06EB8306B042C9D025
:10049000FFF7AEFF0028C4D10020BDE8F88F01208F
:1004A000BDE8F88F4824002010B5202383F311887D
:1004B0001248C3680BB101F097FE0023104A0F48A1
:1004C0004FF47A7101F054FE002383F311880D4C30
:1004D000236813B12368013B2360636813B1636829
:1004E000013B6360084B1B7833B9636823B9022072
:1004F00000F07CFC3223636010BD00BF3424002078
:10050000A9040008782500207024002010B5254B90
:10051000254953F8042F013200D110BD8B42F8D188
:10052000224C234B22689A423AD9224B9B6803F112
:10053000006303F580439A4232D2002000F068FB4A
:100540001D4B0220187000F043FC1C4B1A6C00225B
:100550001A64196E1A66196E596C5A64596E5A6685
:100560005A6E5A6942F080025A615A6922F080023A
:100570005A615A691A6942F000521A611A6922F0E6
:1005800000521A611B6972B60D4A0E4B13601B684C
:100590002268202181F311889D4683F30888104743
:1005A00010BD00BFFC3F00081C40000804400008CC
:1005B000FF3F00082824002070240020003802405B
:1005C00008ED00E0004000082DE9F04F99B0B34C71
:1005D00001902022FF2110A8A66800F043FCB04A39
:1005E0001378A346A3B9AF480121C360117020233B
:1005F00083F31188C3680BB101F0F6FD0023AA4A0A
:10060000A8484FF47A7101F0B3FD002383F31188F9
:10061000019B13B1A54B019A1A60A54AA349019FFA
:100620000292002313704B6099461C461D46984663
:10063000012000F0CDFB002F00F012829B4B1B68C5
:10064000002B40F00D8219B0BDE8F08F0220FFF7BB
:10065000B9FE002840F0FB81019BB9F1000F08BFF3
:100660001F46944B1B88ADF82C3002210BA800F0DC
:100670009FFADDE74FF47A7000F02EFA031E039321
:10068000EADB0220FFF79EFE82460028E4D0039BAF
:10069000581E042800F2DD81DFE800F0030E11147B
:1006A000170018A8052340F8343D042100F080FA13
:1006B00054464FF0000856E004217848F6E704213C
:1006C0007D48F3E704217D48F0E71C24204600F034
:1006D000A1FA04340B9004210BA800F069FA2C2C29
:1006E000F4D1E5E7002DB7D0002CB5D00220FFF7FC
:1006F00069FE0546002800F0AF8101206C4C00F037
:1007000087FA0220207000F063FB4FF000095FFAC7
:1007100089FA504600F08CFA074658B1504600F06E
:1007200097FA09F101090028F1D12C46A9460027C2
:10073000634B97E701230220237000F03BFB3E460A
:10074000DBF808309E4206D2304600F063FA0130F2
:10075000EBD10436F4E7029B00261E70534BA946EA
:100760005E602C46374600F085FB15B1002C18BFA3
:100770000027FFF72FFE5BE7002D3FF46DAF002C45
:100780003FF46AAF029B0220187000F021FB322078
:1007900000F0A2F9B0F1000AC0F25E811AF0030580
:1007A00040F05A81DBF8082006EB0A03934200F27E
:1007B0005381BAF5807F00F24F8155450DDA4FF431
:1007C0007A7000F089F90490049B002BC0F24481F8
:1007D0003C4A049BAB540135EFE7C820FFF7F2FD1C
:1007E0000546002800F038811F2E11D8C6F12004DC
:1007F000544528BF544610AB26F003002246314929
:10080000184400F005FB2246FF212E4800F02AFB89
:100810004FEAAA0A5FFA8AF22A493046FFF7F8FD42
:100820000446002800F01A8106EB8A0605469AE77E
:100830000220FFF7C7FD00283FF40EAFFFF7D8FDF9
:1008400000283FF409AF4FF0000A5346DBF80820B8
:1008500092451CD2BAF11F0F12D8109A01320FD054
:100860002AF0030218A90A4452F8202C0B921846C9
:1008700004220BA900F0A8FB0AF1040A0346E5E7ED
:100880005046039300F0C6F9039B0B90EFE718A8BE
:10089000042140F84C3D00F08BF964E72824002047
:1008A0007425002034240020A904000878250020A5
:1008B00070240020BE3B00082C240020302400209F
:1008C000C03B00087424002018A8002340F8343DE1
:1008D000642100F039F900287FF4BEAE0220FFF752
:1008E00071FD00283FF4B8AE0B9800F0C3F918ABC7
:1008F00043F8480D04211846CDE718A8002340F816
:10090000343D642100F020F900287FF4A5AE0220D8
:10091000FFF758FD00283FF49FAE0B9800F0B8F9A0
:1009200018AB43F8440DE5E70220FFF74BFD002824
:100930003FF492AE00F0B2F918AB43F8400DD9E79E
:100940000220FFF73FFD00283FF486AE0BA91420DC
:1009500000F0AAF9824618A8042140F83CAD00F046
:1009600027F951460BA896E7322000F0B5F8B0F110
:10097000000AFFF671AE1AF0030F7FF46DAEDBF8DC
:1009800008200AEB080393423FF666AE0220FFF709
:1009900019FD00283FF460AE2AF0030AC244D04596
:1009A0003FF4E1AE404600F035F904210A900AA870
:1009B00000F0FEF808F10408F1E74FF47A70FFF751
:1009C00001FD00283FF448AEFFF712FD00283FF478
:1009D000AFAE109B01330CD0082210A90020FFF706
:1009E00017FD00283FF4A4AE2022FF2110A800F03C
:1009F00039FAFFF7EFFC374801F076FB23E6002DCC
:100A00003FF42AAE002C3FF427AE18A8002340F88C
:100A1000343D642100F098F8824600287FF41CAE33
:100A20000220FFF7CFFC00283FF416AE0390FFF73B
:100A3000D1FC41F2883001F057FB0B9800F064FACA
:100A400000F018FA039B57461C461D46F0E5054684
:100A500089E64FF00008FFE52546FDE52C4667E6F0
:100A6000002000F039F80490049B002BFFF6E3AD62
:100A7000012000F09FF9049B213B122B3FF6D8ADDB
:100A800001A252F823F000BF4D06000875060008C9
:100A9000E5060008310600083106000831060008A6
:100AA000790700086909000831080008C90800082A
:100AB000FB08000829090008310600084109000860
:100AC00031060008BB090008670700083106000866
:100AD000FF090008A08601002DE9F34702AE0024BB
:100AE0004FF47A7506F8014D144FDFF858804543EE
:100AF00097F900305A1C5FFA84F901D0A34212D151
:100B000058F8240003680122D3F820A031462B4670
:100B1000D047012807D10A4B9DF8070083F80090C1
:100B200002B0BDE8F0870134032CE1D14FF4FA7034
:100B300001F0DAFA4FF0FF30F2E700BF00240020A6
:100B400098250020143C00082DE9F0474FF47A75F1
:100B5000144FDFF8588006464D43002497F90030C3
:100B60005A1C5FFA84F901D0A34210D158F824002E
:100B700003680422D3F820A031462B46D04704282E
:100B800005D1094B83F800900020BDE8F0870134BF
:100B9000032CE3D14FF4FA7001F0A6FA4FF0FF30C6
:100BA000BDE8F0870024002098250020143C0008B0
:100BB00030B4074B1A78074B53F822402368DD699D
:100BC000054B0A46AC460146204630BC604700BF94
:100BD00098250020143C0008A086010070B501F0A3
:100BE000CFFC094C094E20700025306823788342E1
:100BF00008D901F0BFFC336805440133B5F5804FD7
:100C00003360F2D370BD00BF9925002080250020FD
:100C100001F06CBD00F1006000F580400068704795
:100C200000F10060920000F5804001F0F7BC000088
:100C3000054B1A68054B1B789B1A834202D9104456
:100C400001F098BC002070478025002099250020E5
:100C500038B5074D04462868204401F093FC28B9B4
:100C600028682044BDE8384001F0A4BC38BD00BF6E
:100C70008025002010F0030308D1B0F5007F05D8CF
:100C800000F10050A0F50840006870470020704750
:100C9000014BC058704700BF107AFF1F014B186806
:100CA000704700BF002004E070B52A4B1C68C4F3F5
:100CB0000B03240C63B140F21342934231D040F253
:100CC000194293422FD040F2214293422DD1032367
:100CD000214A0C2505FB03235D6893F9082042F2A5
:100CE00001039C4224D0B4F5805F23D041F201037C
:100CF0009C4221D041F203039C421FD041F20703E2
:100D00009C4208BF3122441E0C44013D0B46A342C5
:100D10001ED215F9016F581C96B1034600F8016CFC
:100D2000F5E70123D4E70223D2E73F220B4DD6E7B4
:100D30003322E3E74122E1E75A22E4E75922E2E7DE
:100D40002C2584421D7001D9981C5A70401A70BD20
:100D50001846FBE7002004E0E43B0008C43B000821
:100D6000124B5A8842F201018A4293B214D0B3F571
:100D7000805F13D041F20102934211D041F203028D
:100D800093420FD041F2070293420DD10423084A47
:100D900002EB8303D87870470023F8E70123F6E7D6
:100DA0000223F4E70323F2E700207047002004E069
:100DB000D03B0008022802D1044B986170470128FB
:100DC00002BF024B4FF400629A6170470004024078
:100DD000022804D14FF40032034B9A617047012876
:100DE000FCD14FF00062F7E700040240022805D171
:100DF000064A536983F00203536170470128FCD10E
:100E0000024A536983F40063F6E700BF000402401E
:100E100010B50023934203D0CC5CC4540133F9E7EE
:100E200010BD000030B5441E14F9010F0B4660B12F
:100E300093F90050854201F1010106D11AB993F9E5
:100E40000020801A30BD013AEEE7002AF7D11046A3
:100E500030BD000002460346981A13F9011B002911
:100E6000FAD1704702440346934202D003F8011BB3
:100E7000FAE77047024B1A78024B1A70704700BFAE
:100E8000982500200024002038B5184C184D204625
:100E900000F06AFC2946204600F092FC2D681548B7
:100EA000EA6ED2F8043843F00203C2F8043801F0C5
:100EB0001BF91149284600F091FDEA6E0F48D2F85F
:100EC00004380F4923F00203C2F80438A0424FF45B
:100ED000E1330B6001D000F0A5FB0A48A04204D02A
:100EE0000749BDE8384000F09DBB38BD2C2F0020DD
:100EF000F83C000840420F00203D00081C2600205E
:100F000084250020842A002038B50B4B1A780B4B1F
:100F100053F822400A4B9C4205460CD0094B002155
:100F200018461422FFF79EFF056001462046BDE8E3
:100F3000384000F077BB38BD98250020143C0008ED
:100F40002C2F002084250020FEE7000000B59BB078
:100F5000EFF3098168226846FFF75AFFEFF3058334
:100F6000034B9A6B9A6A9A6A9A6A9A6A9B6AFEE734
:100F700000ED00E000B59BB0EFF309816822684600
:100F8000FFF746FFEFF30583044B9A6B9A6A9A6A60
:100F90009A6A9A6A9A6A9B6AFEE700BF00ED00E0CF
:100FA00000B59BB0EFF3098168226846FFF730FF78
:100FB000EFF30583034B5A6B9A6A9A6A9A6A9A6AA4
:100FC0009B6AFEE700ED00E030B5084D0A4491420F
:100FD0000BD011F8013B09245840013CF7D040F3F5
:100FE00000032B4083EA5000F7E730BD2083B8EDC3
:100FF000002304491A465A50C8180833802B42600F
:10100000F9D170479C2500200268436811430160B4
:1010100003B1184770470000024AD36843F0C00389
:10102000D360704700440040024AD36843F0C003D5
:10103000D3607047004800402DE9F041D0F85C646F
:10104000F7683368DA0505469CB20DD5202383F393
:1010500011884FF400710430FFF7D6FF6FF48073EE
:101060003360002383F31188202383F3118805F173
:10107000040814F02F0333D183F31188380615D5F3
:10108000210613D5202383F3118805F1380000F0E1
:1010900027FA002846DA0821281DFFF7B5FF4FF68A
:1010A0007F733B40F360002383F311887A060ED5EB
:1010B00063060CD5202383F31188EA6C2B6D9A42CA
:1010C00002D12B6C002B2FD1002383F31188D5F88C
:1010D0006424D368002B31D01069BDE8F041184773
:1010E000230713D014F0080F0CBF00218021E00764
:1010F00048BF41F02001A20748BF41F0400163070B
:1011000048BF41F480714046FFF77EFFA406736834
:1011100005D595F860142846194000F091FA346816
:10112000A4B2A6E77060BEE727F040073F04102195
:10113000281D3F0CFFF768FFF760C5E7BDE8F081A9
:1011400008B50348FFF778FFBDE8084001F05ABB37
:101150001C26002008B50348FFF76EFFBDE80840D5
:1011600001F050BB842A002010B5094C094A2046E2
:10117000002100F035FA084BC4F85C34074C084AEB
:101180000021204600F02CFA064BC4F85C3410BD58
:101190001C2600201910000800440040842A00206A
:1011A000291000080048004038B5314D037C002963
:1011B00018BF0D46012B0446C0F8645410D12D4BC6
:1011C000984242D12C4B1A6C42F400321A641A6EC7
:1011D00042F400321A661B6E0B21262000F058F8EC
:1011E000264BD4F85C249A422B6802D024498A42C8
:1011F0003BD1244901EB5301B1FBF3F3A988080467
:1012000042BF23F0070003F0070343EA4003936063
:10121000EB8843F040039BB213612B8943F0010339
:101220009BB2536141F4045343F02C03D36001F4A7
:10123000A05100231360B1F5806F136853680CBF91
:101240007F23FF2384F8603438BD0F4B9842C7D109
:10125000094B1A6C42F480221A641A6E42F48022FE
:101260001A661B6E0B212720B8E70849C2E700BFAA
:10127000403C00081C2600200038024000100140BD
:101280000014014000BD0105842A002080DE800298
:1012900000F1604300F01F02400903F561430901BA
:1012A0008000C9B200F1604083F8001300F561408E
:1012B00001239340C0F8803103607047F8B51546AC
:1012C00082680669AA420B46816938BF8568761A2A
:1012D000B542044607D218462A46FFF799FDA3698E
:1012E0002B44A3610DE011D932461846FFF790FD5B
:1012F000AF1B3A46E1683044FFF78AFDE2683A44A2
:10130000A261A3685B1BA3602846F8BD18462A4665
:10131000FFF77EFDE368E4E783682DE9F0410446CA
:1013200093421546266938BF85684069361AB5422A
:101330000F4606D22A46FFF76BFD63692B446361B3
:101340000DE012D93246A5EB0608FFF761FD4246D3
:10135000B919E068FFF75CFDE26842446261A36886
:101360005B1BA3602846BDE8F0812A46FFF750FDCD
:10137000E368E4E710B50A440024C361029B0060FF
:1013800040608460C160816141610261036210BD9F
:1013900008B582694369934201D1826882B9826843
:1013A000013282605A1C42611970426903699A4293
:1013B00001D3C3684361002100F0B2FE002008BDE4
:1013C0004FF0FF3008BD000070B5202304460E46E4
:1013D00083F31188A568A5B1A368A269013BA36046
:1013E000531CA36115782269934224BFE368A3616B
:1013F000E3690BB120469847002383F31188284600
:1014000070BD3146204600F07BFE0028E2DA85F30D
:10141000118870BD2DE9F74F05460F4690469A4654
:10142000D0F81C90202686F311884FF0000B14464C
:1014300064B1224639462846FFF740FF034668B9A3
:101440005146284600F05CFE0028F1D0002383F3CB
:101450001188A8EB040003B0BDE8F08FB9F1000FCC
:1014600003D001902846C847019B8BF31188E41AEA
:101470001F4486F31188DBE7C16081614161C3616C
:101480001144009B0060406082600161036270470C
:10149000F8B504460E461746202383F31188A56845
:1014A000A5B1A368013BA36063695A1C62611E7009
:1014B000236962699A4224BFE3686361E3690BB1FF
:1014C00020469847002080F31188F8BD3946204611
:1014D00000F016FE0028E2DA85F31188F8BD00005E
:1014E000836942699A4210B501D182687AB98268EB
:1014F000013282605A1C82611C7803699A4201D3CE
:10150000C3688361002100F00BFE204610BD4FF040
:10151000FF3010BD2DE9F74F05460F4690469A461D
:10152000D0F81C90202686F311884FF0000B14464B
:1015300064B1224639462846FFF7EEFE034668B9F5
:101540005146284600F0DCFD0028F1D0002383F34B
:101550001188A8EB040003B0BDE8F08FB9F1000FCB
:1015600003D001902846C847019B8BF31188E41AE9
:101570001F4486F31188DBE702684368114301606A
:1015800003B11847704700001430FFF743BF000055
:101590004FF0FF331430FFF73DBF00003830FFF746
:1015A000B9BF00004FF0FF333830FFF7B3BF000082
:1015B0001430FFF709BF00004FF0FF311430FFF780
:1015C00003BF00003830FFF763BF00004FF0FF3269
:1015D0003830FFF75DBF000000207047FFF7C4BD43
:1015E00037B50F4B0360002343608360C360012362
:1015F00004460374154600900B464FF4007200F148
:101600005C011430FFF7B6FE00942B464FF40072D5
:1016100004F5177104F13800FFF72EFF03B030BD59
:10162000543C000810B52023044683F31188FFF7CB
:10163000BBFD02232374002383F3118810BD000037
:1016400038B5C36904460D461BB904210844FFF7A9
:1016500093FF294604F11400FFF79AFE002806DAEA
:10166000201D4FF48061BDE83840FFF785BF38BDCD
:10167000026843681143016003B1184770470000D6
:1016800013B5446BD4F894341A681178042915D131
:10169000217C022912D11979128901238B4013422E
:1016A0000CD101A904F14C0001F076FED4F8944469
:1016B000019B21790246206800F0E0F902B010BDDC
:1016C000143001F0F9BD00004FF0FF33143001F089
:1016D000F3BD00004C3001F0CBBE00004FF0FF33F3
:1016E0004C3001F0C5BE0000143001F0C7BD000051
:1016F0004FF0FF31143001F0C1BD00004C3001F05B
:1017000097BE00004FF0FF324C3001F091BE000058
:10171000D0F8942438B5136819780429054601D007
:10172000012038BD017C0229FAD112795C8901209F
:1017300090400440F4D105F1140001F059FD024637
:101740000028EDD0D5F894544FF480732868697957
:1017500000F082F9204638BD406BFFF7D9BF00008A
:1017600000207047704700007FB5124B03600023D4
:1017700043608360C360012502260F4B0574044655
:101780000290019300F18402294600964FF4807381
:10179000143001F009FD094B0193029400964FF4B7
:1017A000807304F52372294604F14C0001F0D0FD4A
:1017B00004B070BD7C3C0008591700088116000871
:1017C0000B68202282F311880A7903EB82021062EF
:1017D0004A790D3243F822008A7912B103EB820371
:1017E000186202230374C0F89414002383F3118851
:1017F0007047000038B5037F044613B190F85430A9
:10180000ABB9201D01250221FFF732FF04F11400BE
:1018100025776FF0010100F08FFC84F8545004F13B
:101820004C006FF00101BDE8384000F085BC38BDC8
:1018300010B5012104460430FFF71AFF0023237777
:1018400084F8543010BD000038B50446002514302B
:1018500001F0C2FC04F14C00257701F091FD201D40
:1018600084F854500121FFF703FF2046BDE83840BB
:10187000FFF74EBF90F85C3003F06003202B19D1C6
:1018800090F85D20212A0AD0222A4FF000030ED0C2
:10189000202A0FD1084A02650722426504E0064B60
:1018A00003650723436500238365012070470365B3
:1018B0004365F9E70020704701240020D0F89434F4
:1018C00037B51A681178042904461AD1017C022917
:1018D00017D11979128901238B40134211D100F1DC
:1018E0004C05284601F00CFE58B101A9284601F02C
:1018F00053FDD4F89444019B21790246206800F0FE
:10190000BDF803B030BD000000EB8103F7B51C6AE1
:1019100005460E46F4B1202383F3118805EB8607B4
:10192000201D0821FFF7A4FEFB685B691B684C348F
:1019300013B1204601F03EFD01A9204601F02CFD27
:10194000024648B1019B3146284600F097F8002333
:1019500083F3118803B0F0BDFB685A691268002A4E
:10196000F5D01B8A013B1340F1D105F15C02EAE797
:101970000D3138B550F82140DCB1202383F31188B4
:10198000D4F894241368527903EB8203DB689B69D3
:101990005D6845B104216018FFF76AFE294604F12D
:1019A000140001F02FFC2046FFF7B2FE002383F362
:1019B000118838BD7047000000F0DCBF01230370C0
:1019C0000023436000F1240200F1380142F8043B97
:1019D0008A421361FAD103814381704738B50446C6
:1019E000202383F3118800254160C56005614561AE
:1019F0008561C561056200F0CDFF0223237085F388
:101A0000118838BD70B500EB810305465069DA6076
:101A10000E46144618B110220021FFF723FAA069E0
:101A200018B110220021FFF71DFA31462846BDE803
:101A3000704001F079B80000028902F001020281D1
:101A4000428902F001024281002202614261826108
:101A5000C261026201F0FCB8F0B400EB8104478976
:101A6000E4680125A4698D403D434581236000233E
:101A7000A2606360F0BC01F017B90000F0B400EBA5
:101A800081040789E468012564698D403D4305812F
:101A900023600023A2606360F0BC01F091B90000F4
:101AA00070B50223002504460370A0F8645080F846
:101AB000665080F8675005814581C56005614561C4
:101AC0008561C561056280F84C5000F0C9FF63680C
:101AD0001B6823B129462046BDE87040184770BDF9
:101AE000436802781B6880F86820052202700BB1F9
:101AF0000421184770470000436890F868201B686D
:101B000002700BB1052118477047000090F84C3067
:101B100070B5044613B1002380F84C3004F15C0228
:101B2000204601F0B7F863689B6863BB94F85C508B
:101B300015F0600615D194F85D3005F07F0545EA93
:101B4000032540F202339D4200F00E815BD8022D46
:101B500000F0DC803FD8002D00F08780012D00F0E0
:101B6000CF800021204601F001FB0021204601F03A
:101B7000F3FA63681B6813B10621204698470623D1
:101B800084F84C3070BD204698470028CED094F899
:101B9000632094F8623043EA0223626D934238BFB7
:101BA000636594F95C30656D002B4FF0200380F283
:101BB000FD80002D00F0EC80092284F84C2083F396
:101BC00011880021636D226D2046FFF757FF002327
:101BD00083F3118870BDB5F5817F00F0B180B5F554
:101BE000407F49D0B5F5807FBBD194F85E30012BA2
:101BF000B7D1B4F8643023F00203A4F8643026654A
:101C00006665A665C3E740F201639D421ED8B5F53F
:101C1000C06F3BD2B5F5A06FA3D1B4F85C30B3F57B
:101C2000A06F0ED194F85E3084F86630204600F044
:101C30006FFF63681B6813B1012120469847032397
:101C40002370002323656365A365A0E7B5F5106FD6
:101C500032D040F602439D4252D0B5F5006F80D19C
:101C600004F167032365012324E004F16403236581
:101C700002236365A5658AE794F85E30012B7FF443
:101C800070AFB4F8643043F00203B6E794F8612013
:101C9000616894F860304D6894F85F1043EA02235D
:101CA000204694F85E20A84700283FF45AAF4368C6
:101CB000236503686365A4E72378042B10D12023F0
:101CC00083F311882046FFF7B7FE86F31188636817
:101CD00084F867601B68032121700BB12046984788
:101CE00094F85E30002BACD084F867300423237066
:101CF00063681B68002BA4D0022120469847A0E708
:101D0000374B23650223636500239DE794F8601039
:101D100011F0800F204601F00F010ED000F0ACFF53
:101D2000012806D002287FF41CAF2E4B2365606586
:101D300067E72D4B2365656563E700F08FFFEFE7ED
:101D400094F85E30002B7FF40CAF94F8603013F001
:101D50000F013FF476AF1A06204602D501F01AFAB9
:101D60006FE701F00DFA6CE794F85E30002B7FF41A
:101D7000F8AE94F8603013F00F013FF462AF1B0629
:101D8000204602D501F0F2F95BE701F0E5F958E7EA
:101D9000142284F84C2083F311882B462A462946C6
:101DA0002046FFF759FE85F3118870BD5DB11522FD
:101DB00084F84C2083F311880021636D226D204646
:101DC000FFF74AFE03E70B2284F84C2083F31188C7
:101DD0002B462A4629462046FFF750FEE3E700BF80
:101DE000AC3C0008A43C0008A83C000838B590F8BA
:101DF0004C300446152B29D8DFE803F03E2828286C
:101E000028283E28280B2939282828282828282847
:101E10003E3E90F8631090F86220436D42EA012242
:101E20009A4214D9C268128AB3FBF2F502FB153547
:101E30006DB9202383F311882B462A462946FFF7E4
:101E40001DFE85F311880A2384F84C3038BD142315
:101E500084F84C30202383F3118800231A46194656
:101E60002046FFF7F9FD002383F3118838BD836D09
:101E700003B198470023E7E7002101F077F900213B
:101E8000204601F069F963681B6813B106212046FA
:101E900098470623D8E7000090F84C20152A38B55B
:101EA000044622D80123934040F6416213421DD1DB
:101EB00013F480150FD19B0217D50B2380F84C30FB
:101EC000202383F311882B462A462946FFF7D6FDA7
:101ED00085F3118838BDC3689B695B682BB9836D36
:101EE00003B19847002384F84C3038BD002101F03D
:101EF0003DF90021204601F02FF963681B6813B1FA
:101F00000621204698470623EDE70000024B0022F9
:101F10001B605B609A607047EC2E00200023037406
:101F20008268054B1B6899689142FBD25A6803602E
:101F30004260106058607047EC2E002008B52023E6
:101F400083F31188037C032B05D0042B0DD02BB910
:101F500083F3118808BD436900221A604FF0FF33F4
:101F60004361FFF7DBFF0023F2E790E80C001A6003
:101F700002685360F2E70000002303748268054B97
:101F80001B6899689142FBD85A68036042601060F0
:101F900058607047EC2E0020054B196908741868CA
:101FA00002681A605360186101230374FEF7ACB92C
:101FB000EC2E002030B54B1C87B005460A4C10D0E3
:101FC00023690A4A01A800F0D3F82846FFF7E4FF86
:101FD000049B13B101A800F007F92369586907B001
:101FE00030BDFFF7D9FFF8E7EC2E00203D1F0008B9
:101FF00038B50C4D41612B6981689A68914204465D
:1020000003D8BDE83840FFF789BF1846FFF786FFC1
:1020100001232C61014623742046BDE83840FEF7B9
:1020200073B900BFEC2E0020044B1A681B6990683E
:102030009B68984294BF002001207047EC2E00203E
:1020400010B5084C236820691A6822605460012288
:1020500023611A74FFF790FF01462069BDE8104024
:10206000FEF752B9EC2E0020826002220274002298
:10207000427470478368A3F17C0243F80C2C026918
:1020800043F83C2C426943F8382C074A43F81C2C8F
:10209000C26843F8102C022203F8082C002203F82F
:1020A000072CA3F1180070472103000810B5202366
:1020B00083F31188FFF7DEFF00210446FFF798FF46
:1020C000002383F31188204610BD0000024B1B69DA
:1020D00058610F20FFF760BFEC2E0020202383F310
:1020E0001188FFF7F3BF000008B50146202383F3F2
:1020F00011880820FFF75EFF002383F3118808BDD5
:1021000049B1064B42681B6918605A60136043600E
:102110000420FFF74FBF4FF0FF307047EC2E002038
:102120000368984206D01A680260506059611846E8
:10213000FFF7F4BE7047000038B504460D4620682E
:10214000844200D138BD036823605C604561FFF7BD
:10215000E5FEF4E7054B03F114025A619A614FF072
:10216000FF32DA6100221A62704700BFEC2E0020B5
:10217000F8B503611A4BC2605C6A1A4B1A46022911
:1021800052F8145F38BF0221954206461F460AD115
:10219000586198611C620560456081600819BDE85E
:1021A000F84001F0CFB9186AAB68241A0C1902D3B1
:1021B000E41A2D6804E09C4202D2204401F0D2F9D6
:1021C000AB689C42F4D86B68736035601E606E60CB
:1021D000B460A9684FF0FF33091BA960FB61F8BD2B
:1021E000000C0040EC2E002010B41A4C234653F88B
:1021F000141F814210D0416802680A600268516071
:102200009A424FF00001C16003D0936881680B448B
:1022100093605DF8044B70470A68626100209A423F
:102220005360C86003D15DF8044B01F095B9936821
:10223000886803449360084A206A526A121A9342DB
:10224000E7D9991A012998BF931C18445DF8044BEB
:1022500001F088B9EC2E0020000C004000207047EF
:10226000FEE70000704700004FF0FF3070470000AD
:10227000022906D0032906D00129064818BF0020EC
:10228000704705487047032A9ABF044800EBC20014
:10229000002070477C3D0008303D000808240020E5
:1022A00070B59AB001AD064608462946144600F0BE
:1022B00095F82846FEF7CEFDC0B2431C5B0086E8C9
:1022C0001800237003236370002302341946DAB226
:1022D000904204F1020401D81AB070BDEA5C04F81F
:1022E000022C04F8011C0133F1E7000008B520239B
:1022F00083F311880348FFF7E1FA002383F3118881
:1023000008BD00BF2C2F002010B50446052916D8A3
:10231000DFE801F016150316161D202383F311883C
:102320000E4A0121FFF76EFB20460D4A0221FFF7FE
:1023300069FB0C48FFF788FA002383F3118810BD6E
:10234000202383F311880748FFF754FAF4E720238A
:1023500083F311880348FFF76BFAEDE7B03C000800
:10236000D43C00082C2F002038B50C4D0C4C0D49E6
:102370002A4604F10800FFF793FF05F1CA0204F1B1
:1023800010000949FFF78CFF05F5CA7204F1180027
:102390000649BDE83840FFF783BF00BFF433002093
:1023A00008240020003D00080A3D0008153D0008F3
:1023B00070B5044608460D46FEF74CFDC6B22046F1
:1023C000013403780BB9184670BD32462946FEF732
:1023D00029FD0028F3D1012070BD00002DE9F84F40
:1023E00005460C46FEF736FD2C49C6B22846FFF7D7
:1023F000DFFF08B10436F6B229492846FFF7D8FFB7
:1024000008B11036F6B2632E0DD8DFF89090DFF8E1
:1024100090A0DFF89880DFF898B0224F2E7846B968
:102420002670BDE8F88F29462046BDE8F84F01F038
:10243000BDBB252E2DD1072249462846FEF7F2FCCA
:1024400050B93B6823607B6863603B892381BB7A1A
:10245000A37207350B34E1E7082251462846FEF700
:10246000E1FCB0B9104BA21C13F8011F09095B4530
:1024700011F8081002F8021C197801F00F0102F19E
:10248000020211F8081002F8031CEDD118340835C7
:10249000C4E7267001350134C0E700BF9C3D000849
:1024A000153D0008A43D00080F7AFF1FB03D00084D
:1024B0001B7AFF1FBFF34F8F024AD368DB03FCD4A4
:1024C000704700BF003C024008B5094B1B7873B948
:1024D000FFF7F0FF074B1A69002ABFBF064A5A6090
:1024E00002F188325A601A6822F480621A6008BDCC
:1024F00052360020003C02402301674508B50B4BD3
:102500001B7893B9FFF7D6FF094B1A6942F00042D6
:102510001A611A6842F480521A601A6822F48052D2
:102520001A601A6842F480621A6008BD52360020B0
:10253000003C0240172870B513D80B4A0B4C137897
:1025400063B90B4E4FF0006144F8231056F8235046
:102550000133182B2944F7D10123137054F82000BC
:1025600070BD002070BD00BFB4360020543600207E
:10257000C43D0008014B53F820007047C43D0008DB
:1025800018207047172810B5044601D9002010BD47
:10259000FFF7D0FF064B53F824301844C21A0BB98A
:1025A000012010BD12680132F0D1043BF6E700BFF4
:1025B000C43D0008172810B5044629D8FFF77AFF54
:1025C000FFF782FF1349F323CB600C23B0FBF3F238
:1025D00003FB1200D30143EAC003DBB243F40073F0
:1025E00043F002030B610B6943F480330B61FFF787
:1025F00061FF2046FFF79EFF074B53F8241000F0C1
:10260000DDF8FFF77BFF2046BDE81040FFF7BABFBB
:10261000002010BD003C0240C43D00082DE9F843F5
:1026200012F00103154640D18218B2F1026F3CD27C
:102630002C4B1B6813F0010337D02B4CFFF744FFE2
:10264000F323E360FFF736FF40F20127032D01D9A2
:10265000830713D0244C0F46401A40F20118EB1B9D
:102660000B44012B00EB0706236924D823F0010358
:102670002361FFF743FF0120BDE8F883236923F4BA
:102680004073236123693B43236151F8046B066067
:10269000BFF34F8FFFF70EFF03689E4208D02369F8
:1026A00023F001032361FFF729FF0020BDE8F88331
:1026B000043D0430CAE723F440732361236943EAED
:1026C00008032361B94637F8023B3380BFF34F8FCD
:1026D000FFF7F0FE3688B9F80030B6B2B342BED08C
:1026E000DDE700BF00380240003C0240084908B561
:1026F0000B7828B153B9FFF7E7FE01230B7008BD33
:1027000023B1BDE808400870FFF7F8BE08BD00BF60
:102710005236002010B50244064B0439D2B2904222
:1027200000D110BD441C00B253F8200041F8040F42
:10273000E0B2F4E750280040104B30B51C6F240481
:1027400007D41C6F44F400741C671C6F44F40044ED
:102750001C670B4C236843F4807323600244094BCD
:102760000439D2B2904200D130BD441C00B251F8BD
:10277000045F43F82050E0B2F4E700BF00380240A5
:10278000007000405028004007B5012201A9002038
:10279000FFF7C0FF019803B05DF804FB13B50446D2
:1027A000FFF7F2FFA04206D002A9012241F8044D32
:1027B0000020FFF7C1FF02B010BD0000704700000D
:1027C000034B1B689B0042BF024B01221A707047EB
:1027D00074380240B5360020014B1878704700BFAE
:1027E000B5360020064A536823F001035360EFF327
:1027F0000983683383F30988002383F311887047C2
:1028000030EF00E010B5202383F31188104B5B6894
:1028100013F4006318D0F1EE103AEFF309844FF08F
:10282000807344F84C3C0B4BDB6844F8083CA4F143
:10283000680383F30988FFF7F7FB18B1064B44F8E8
:10284000503C10BD054BFAE783F3118810BD00BF63
:1028500000ED00E030EF00E0310300083403000831
:1028600070470000FEE70000084A094B09498B4207
:1028700004D3094A0021934205D3704752F8040F4C
:1028800043F8040BF3E743F8041BF4E7D43F0008D4
:10289000403900204039002040390020036F30B516
:1028A00000229D68C46E11464FF0FF3004EB4213C6
:1028B00001329542C3F80019C3F81019C3F808098A
:1028C000C3F8001BC3F8101BC3F8080BEED24FF07F
:1028D0000113C4F81C3830BD890141F020010161A9
:1028E00003699B06FCD4122000F0C8BE204B03EB0A
:1028F00080022DE9F047D2F80CE0DD6EDEF81420FE
:10290000461CD2F800C005EB063605EB40185168AE
:1029100061450BD3D5F83428012303FA00F022EAED
:102920000000C5F834081846BDE8F087BEF810402E
:10293000ACEB0103A34228BF2346D8F81849A4B240
:10294000B3EB840F10D894681F46A4F1040959F81A
:1029500004AFC6F800A0042F01D9043FF7E71C44D8
:102960000B4494605360D2E70020BDE8F08700BFBD
:10297000B836002010B5054C2046FFF71FF84FF081
:10298000A043E366024B236710BD00BFB8360020AA
:10299000483E00080378012B70B5054650D12A4BFC
:1029A000C46E98421BD1294B5A6B42F080025A6385
:1029B0005A6D42F080025A655A6D5A6942F080029F
:1029C0005A615A6922F080025A610E2143205B69E4
:1029D000FEF75EFC1E4BE3601E4BC4F8003800237C
:1029E000C4F8003EC0232360EE6E4FF40413A363CB
:1029F0003369002BFCDA012333610C2000F03EFE2A
:102A00003369DB07FCD4122000F038FE3369002B59
:102A1000FCDA0026A6602846FFF740FF6B68C4F882
:102A20001068DB68C4F81468C4F81C684BB90A4B1A
:102A3000A3614FF0FF336361A36843F00103A36018
:102A400070BD064BF4E700BFB836002000380240E6
:102A50004014004003002002003C30C0083C30C05D
:102A6000F8B5C46E054600212046FFF735FF296FF3
:102A700000234FF001128F68C4F834384FF000661D
:102A8000C4F81C284FF0FF3004EB431201339F427F
:102A9000C2F80069C2F8006BC2F80809C2F8080B56
:102AA000F2D20B68EA6E6B676362102313611669DA
:102AB00016F01006FBD1122000F0E0FDD4F800382B
:102AC00023F4FE63C4F80038A36943F4402343F0C1
:102AD0001003A3610923C4F81038C4F814380A4B52
:102AE000EB604FF0C043C4F8103B084BC4F8003B08
:102AF000C4F81069C4F800396B6F03F1100243F495
:102B000080136A67A362F8BD243E0008408000106D
:102B1000C26E90F86610D2F8003823F4FE6343EAE0
:102B20000113C2F8003870472DE9F0410EB200EBF6
:102B300086080D46D8F80C100F6807F00303022B27
:102B400050D0032B50D03D4A3D4F012B18BF1746A4
:102B5000C46E4FEA451E04EB0E030022C3F8102B8F
:102B60008A6905F1100C002A40D04A8A05F1580301
:102B70005B013A43E2500123D4F81C2803FA0CF31A
:102B80001343A6444A69C4F81C380023CEF8103910
:102B900005F13F03002A39D00A8A898B920801295E
:102BA00088BF4A43416F04EB8303561841EA02424F
:102BB000466729465A602046FFF78EFED8F80C304B
:102BC0001B8A43EA85531F4305F148035B01E75025
:102BD0000123D4F81C2803FA05F51543C4F81C5842
:102BE000BDE8F081174FB3E7174FB1E704EB461389
:102BF000D3F8002B22F40042C3F8002BD4F81C2891
:102C0000012303FA0CF322EA0303BAE704EB83037C
:102C10000E4A5A6004EB461629462046FFF75CFE32
:102C2000D6F8003923F40043C6F80039D4F81C382C
:102C3000012202FA05F523EA0505CFE7008000101E
:102C4000008004100080081000800C1000040002B6
:102C5000026F12684267FFF721BE00005831C36E51
:102C600049015B5813F4004004D013F4001F14BF53
:102C700001200220704700004831C36E49015B58B3
:102C800013F4004004D013F4001F14BF01200220ED
:102C90007047000000EB8101CB68196A0B68136074
:102CA0004B6853607047000000EB810330B5DD686E
:102CB000AA691368D36019B9402B84BF40231360FD
:102CC0006B8A1468C26E1C44013CB4FBF3F463438A
:102CD000033323F0030302EB411043EAC44343F000
:102CE000C043C0F8103B2B6803F00303012B09B26B
:102CF0000ED1D2F8083802EB411013F4807FD0F8DF
:102D0000003B14BF43F0805343F00053C0F8003B36
:102D100002EB4112D2F8003B43F00443C2F8003BFF
:102D200030BD00002DE9F041244DEE6E06EB40135E
:102D30000446D3F8087BC3F8087B38070AD5D6F8D1
:102D40001438190706D505EB84032146DB682846AD
:102D50005B689847FA072FD5D6F81438DB072BD5D0
:102D600005EB8403D968CCB98B69488A5E68B6FBE9
:102D7000F0F200FB12628AB91868DA6890420DD24C
:102D8000121A83E81400202383F311880B4821468C
:102D9000FFF78AFF84F31188BDE8F081012303FA6D
:102DA00004F26B8923EA02036B81CB6823B12146CD
:102DB0000248BDE8F0411847BDE8F081B836002070
:102DC00000EB810370B5DD68C36E6C692668E66050
:102DD0004A0156BB1A444FF40020C2F810092A6871
:102DE00002F00302012A0AB20ED1D3F8080803EB5D
:102DF000421410F4807FD4F8000914BF40F08050D2
:102E000040F00050C4F8000903EB4212D2F8000968
:102E100040F00440C2F80009D3F83408012202FA55
:102E200001F10143C3F8341870BD19B9402E84BFB5
:102E30004020206020682E8A841940F00050013C18
:102E40001A44B4FBF6F440EAC440C6E7F8B50446B9
:102E50001E48C56E05EB4413D3F80869C3F808692A
:102E6000F10717D5D5F81038DA0713D500EB84032E
:102E7000D9684B691F68DA68974218D2D21B0027BD
:102E80001A605F60202383F311882146FFF798FFC3
:102E900087F31188330617D5D5F834280123A340CA
:102EA000134211D02046BDE8F840FFF71FBD0123B3
:102EB00003FA04F2038923EA020303818B68002BDF
:102EC000E8D021469847E5E7F8BD00BFB8360020B6
:102ED000A0482DE9F84FC56E6E69AB691E4016F427
:102EE000805F6E61044605D0FEF7DAFDBDE8F84F5D
:102EF000FFF788BC002E12DAD5F8003E95489B07F4
:102F00001EBFD5F8003E23F00303C5F8003ED5F8F8
:102F1000043823F00103C5F80438FEF7EDFD37054A
:102F200002D58C48FEF7DCFDB0040CD5D5F8083886
:102F300013F0060FEB6823F470530CBF43F41053E7
:102F400043F4A053EB60310704D56368DB680BB131
:102F500080489847F2026FD4B3020CD5D4F86C8045
:102F6000DFF8F0A100274FF00109236F9B68F9B249
:102F70008B4280F09C80F70619D5E16E0A6AC2F395
:102F80000A1702F00F0302F4F012B2F5802F00F0DE
:102F9000B680B2F5402F0AD104EB830301F58051CE
:102FA000DB68186A00231A469F4240F09C80330376
:102FB000D5F818481DD5E70302D50020FFF7B2FE6B
:102FC000A50302D50120FFF7ADFE600302D5022064
:102FD000FFF7A8FE210302D50320FFF7A3FEE202BC
:102FE00002D50420FFF79EFEA30202D50520FFF7BD
:102FF00099FE77037FF57AAFE60702D50020FFF749
:1030000025FFA50702D50120FFF720FF600702D5A5
:103010000220FFF71BFF210702D50320FFF716FF51
:10302000E20602D50420FFF711FFA3067FF55EAF8D
:103030000520FFF70BFF59E7D4F86C80DFF814A1E7
:1030400000274FF00109236F9B685FFA87FB5B4500
:1030500082D308EB4B13D3F8002902F44022B2F5D7
:10306000802F22D1D3F80029002A1EDAD3F80029B4
:1030700042F09042C3F80029D3F80029002AFBDB74
:103080005946E06EFFF728FC228909FA0BF322EA81
:103090000303238104EB8B03DB689B6813B1594660
:1030A000504698475846FFF721FC0137CBE708EB1D
:1030B0004112D2F8003B03F44023B3F5802F10D126
:1030C000D2F8003B002B0CDA628909FA01F322EAFC
:1030D0000303638104EB8103DB68DB680BB15046BB
:1030E0009847013741E79C0708BF0A68072B98BF3C
:1030F000027003F101039CBF120A013054E702334E
:1031000004EB830201F58051526890690268D0F89F
:1031100008C04068A2EB000E0022104697420AD178
:1031200004EB830463689B699A683A449A605A681E
:1031300017445F603BE712F0030F08BF086896452D
:1031400088BF8CF8000002F1010284BF000A0CF174
:10315000010CE3E7B8360020C36E03EB4111D1F850
:10316000003B43F40013C1F8003B7047C36E03EB10
:103170004111D1F8003943F40013C1F80039704708
:10318000C36E03EB4111D1F8003B23F40013C1F8E7
:10319000003B7047C36E03EB4111D1F8003923F4B3
:1031A0000013C1F80039704730B5039C0172043335
:1031B00004FB0325C361049B03630021059B00609E
:1031C0004060C16042610261856104624262816265
:1031D000C162436330BD00000022416A4161016168
:1031E000C2608262C2626FF00101FEF7A5BF0000FB
:1031F00003694269934203D1C2680AB10020704753
:10320000181D704703691960C2680132C260C26943
:10321000134482690361934224BF436A036100211E
:10322000FEF77EBF38B504460D46E3683BB16269E0
:10323000131D1268A3621344E362002038BD237A91
:1032400033B929462046FEF75BFF0028EDDA38BD8A
:103250006FF00100FBE70000C368C269013BC36077
:103260004369134482694361934224BF436A4361C3
:1032700000238362036B03B11847704770B52023A6
:10328000044683F31188866A3EB9FFF7CBFF0546F3
:1032900018B186F31188284670BDA36AE26A13F854
:1032A000015BA362934202D32046FFF7D5FF0023C0
:1032B00083F31188EFE700002DE9F84F04460E462E
:1032C00090469946202787F311880025AA46D4F80E
:1032D00028B0BBF1000F09D149462046FFF7A2FFF5
:1032E00020B18BF311882846BDE8F88FA16AE36A04
:1032F000A8EB050B5B1A9B4528BF9B46BBF1400F13
:103300001BD9334601F1400251F8040B43F8040B7A
:103310009142F9D1A36A40334036A3624035A26A94
:10332000E36A9A4202D32046FFF796FF8AF3118898
:103330004545D8D287F31188C9E730465A46FDF78C
:1033400067FDA36A5B445E44A3625D44E7E7000057
:1033500010B5029C0172043303FB0421C3610023F6
:103360008362C362039B0363049B00604060C4608C
:1033700042610261816104624262436310BD0000E8
:10338000026AC260426A4261026100228262C262D3
:103390006FF00101FEF7D0BE436902699A4203D182
:1033A000C2680AB100207047184650F8043B0B6011
:1033B00070470000C368C2690133C36043691344A6
:1033C00082694361934224BF436A43610021FEF74F
:1033D000A7BE000038B504460D46E3683BB123693B
:1033E0001A1DA262E2691344E362002038BD237A09
:1033F00033B929462046FEF783FE0028EDDA38BDB2
:103400006FF00100FBE7000003691960C268013A30
:10341000C260C269134482690361934224BF436A54
:10342000036100238362036B03B1184770470000F8
:1034300070B5202304460E4683F31188856A35B99A
:103440001146FFF7C7FF10B185F3118870BDA36A5D
:103450001E70A36AE26A01339342A36204D3E16956
:1034600020460439FFF7D0FF002080F3118870BD9B
:103470002DE9F84F04460D4691469A464FF0200834
:1034800088F311880026B346A76A4FB951462046F3
:10349000FFF7A0FF20B187F311883046BDE8F88F11
:1034A000A06AE76AA9EB06033F1A9F4228BF1F469E
:1034B000402F1BD905F1400355F8042B40F8042B8D
:1034C0009D42F9D1A36A4033A3624036A26AE36AFF
:1034D0009A4204D3E16920460439FFF795FF8BF344
:1034E00011884E45D9D288F31188CDE729463A464E
:1034F000FDF78EFCA36A3B443D44A3623E44E5E7EE
:10350000026943699A4203D1C3681BB918467047E0
:103510000023FBE7836A002BF8D0043B9B1AF5D00D
:103520001360C368013BC360C3691A4483690261C5
:103530009A4224BF436A0361002383620123E5E7C3
:1035400000F042B9034B002258631A610222DA608C
:10355000704700BF000C0040014B0022DA6070474A
:10356000000C0040014B5863704700BF000C004046
:10357000FEE7000010B5174CFEF7C8FCFEF7EAFDA9
:10358000802215492046FEF76FFD012344F8180CF0
:103590000374124B124AD96821F4E0610904090C42
:1035A0000A431049DA60CA6842F08072CA600E4964
:1035B0000A6842F001020A601022DA77202283F8BA
:1035C0002220002383F3118862B60848BDE810402A
:1035D000FEF76CBD142F0020543E000800ED00E003
:1035E0000003FA05F0ED00E0001000E05C3E00088A
:1035F0002DE9F84F1F4CDFF88090656904F114073E
:103600004FF00008D9F82430266AAA689E1B96421B
:103610001DD34FF0200AAA68236AD5F80CB01344D2
:1036200023622B68BB425F60A6EB02066361C5F8AC
:103630000C8001D1FFF790FF88F311882869D847E3
:103640008AF311886569AB689E42E4D2DAE7626961
:10365000BA420CD0916823628E1B9660A86802283B
:103660002CBF1818981CBDE8F84FFFF77BBFBDE8CA
:10367000F88F00BFEC2E0020000C0040034B59686F
:103680005A68521A9042FBD8704700BF001000E001
:103690004B6843608B688360CB68C3600B69436190
:1036A0004B6903628B6943620B68036070470000DB
:1036B00008B5274B27481A6940F2FF710A431A617F
:1036C0001A6922F4FF6222F007021A611A691A6B62
:1036D0000A431A631A6D0A431A651F4A1B6D114685
:1036E000FFF7D6FF1D4802F11C01FFF7D1FF1C4870
:1036F00002F13801FFF7CCFF1A4802F15401FFF73D
:10370000C7FF194802F17001FFF7C2FF174802F125
:103710008C01FFF7BDFF164802F1A801FFF7B8FFC3
:10372000144802F1C401FFF7B3FF134802F1E001AE
:10373000FFF7AEFF114802F1FC01FFF7A9FF1048A7
:1037400002F58C71FFF7A4FFBDE8084000F0A8B8AF
:1037500000380240000002407C3E000800040240A5
:1037600000080240000C0240001002400014024019
:1037700000180240001C02400020024000240240C9
:103780000028024008B500F0FFF9FFF7F3FEFFF74D
:1037900017F8BDE80840FEF7E7BD000070470000DD
:1037A000084B1A69920710B508D500241C61202324
:1037B00083F31188FFF71CFF84F31188BDE81040E4
:1037C000FFF720B8000C0040104B1A6C42F00802C2
:1037D0001A641A6E42F008021A660D4A1B6E93684C
:1037E00043F0080393600B4B53229A624FF0FF3271
:1037F000DA6200229A615A63DA605A6001225A61E1
:1038000008211A603220FDF743BD00BF0038024096
:10381000002004E0000C00401F4B1A696FEA42527E
:103820006FEA52521A611A69C2F30A021A614FF022
:10383000FF301A695A69586100215A6959615A69F9
:103840001A6A62F080521A621A6A02F080521A6290
:103850001A6A5A6A58625A6A59625A6A1A6C42F06B
:1038600080521A641A6E42F080521A661A6E0B4A1F
:10387000106840F480701060186F00F44070B0F56C
:10388000007F1EBF4FF4803018671967536823F418
:103890000073536000F058B90038024000700040D7
:1038A000324B4FF080521A64314A4FF4404111605C
:1038B0001A6842F001021A601A689207FCD59A68E9
:1038C00022F003029A60294B19469A6812F00C0202
:1038D000FBD1186800F0F90018609A601A6842F489
:1038E00080321A600B689B03FCD54B6F43F00103D9
:1038F0004B671E4B5A6F9007FCD51E4A5A601A68D8
:1039000042F080721A601A4A53685904FCD5174B6A
:103910001A689201FCD5184A9A600322C3F88C20D9
:10392000164B1A68164B9A42164B1BD1164A116851
:10393000164A914216D140F205121A600B4B9A6852
:1039400042F002029A609A6802F00C02082AFAD148
:103950005A6C42F480425A645A6E42F480425A666B
:103960005B6E704740F20572E7E700BF0038024027
:10397000007000401854400700948838002004E08C
:1039800011640020003C024000ED00E041C20F4104
:10399000084A08B5536911680B4003F001035361ED
:1039A00023B1054A13680BB150689847BDE8084039
:1039B000FEF728BF003C01409C250020084A08B5BE
:1039C000536911680B4003F00203536123B1054AA8
:1039D00093680BB1D0689847BDE80840FEF712BF66
:1039E000003C01409C250020084A08B55369116835
:1039F0000B4003F00403536123B1054A13690BB173
:103A000050699847BDE80840FEF7FCBE003C014005
:103A10009C250020084A08B5536911680B4003F043
:103A20000803536123B1054A93690BB1D0699847E4
:103A3000BDE80840FEF7E6BE003C01409C250020A2
:103A4000084A08B5536911680B4003F0100353612D
:103A500023B1054A136A0BB1506A9847BDE8084084
:103A6000FEF7D0BE003C01409C250020174B10B54E
:103A70005C691A68144004F478725A61A30604D58C
:103A8000134A936A0BB1D06A9847600604D5104A6E
:103A9000136B0BB1506B9847210604D50C4A936BFE
:103AA0000BB1D06B9847E20504D5094A136C0BB1F2
:103AB000506C9847A30504D5054A936C0BB1D06CA4
:103AC0009847BDE81040FEF79DBE00BF003C014096
:103AD0009C2500201A4B10B55C691A68144004F448
:103AE0007C425A61620504D5164A136D0BB1506DC4
:103AF0009847230504D5134A936D0BB1D06D9847B1
:103B0000E00404D50F4A136E0BB1506E9847A10420
:103B100004D50C4A936E0BB1D06E9847620404D55D
:103B2000084A136F0BB1506F9847230404D5054A18
:103B3000936F0BB1D06F9847BDE81040FEF762BE9F
:103B4000003C01409C250020062108B50846FDF7F1
:103B50009FFB06210720FDF79BFB06210820FDF7B0
:103B600097FB06210920FDF793FB06210A20FDF7AC
:103B70008FFB06211720FDF78BFB06212820BDE8CF
:103B80000840FDF785BB000008B5FFF745FEFDF7CF
:103B90002FFAFDF723FDFDF70FFFFDF7E3FDFFF71C
:103BA000FDFDBDE80840FFF7CBBC0000034611F85F
:103BB000012B03F8012B002AF9D1704712101213C0
:103BC0001211000053544D3332463F3F3F00000076
:103BD000012033000010410101105A010310590166
:103BE0000710310100000000C43B00083F00000046
:103BF00013040000203C00083F00000019040000EE
:103C00002A3C00083F00000021040000343C00086A
:103C10003F0000002C2F00201C260020842A0020BA
:103C200053544D3332463430780053544D3332467A
:103C30003432780053544D333246343436585800B9
:103C400000960000000000000000000000000000DE
:103C50000000000000000000A515000891150008F4
:103C6000CD150008B9150008C5150008B1150008E4
:103C70009D15000889150008D915000800000000EE
:103C8000DD160008C916000805170008F11600081F
:103C9000FD160008E9160008D5160008C116000830
:103CA0006117000800000000010000000000000093
:103CB0000200000000000000091900087119000846
:103CC00040004000C4330020D43300200200000034
:103CD000000000000300000000000000B51900080B
:103CE0000000000010000000E4330020000000008D
:103CF0000100000000000000B836002001010200B1
:103D00004172647550696C6F740025424F41524492
:103D1000252D424C002553455249414C25000000B9
:103D2000092300087122000875180008ED22000818
:103D300043000000383D000809024300020100C0B2
:103D400032090400000102020100052400100105EF
:103D50002401000104240202052406000107058253
:103D6000030800FF09040100020A00000007050122
:103D70000240000007058102400000001200000020
:103D8000843D000812011001020000400912415751
:103D900000020102030100000403090425424F410F
:103DA0005244250044726F74656B503350726F003B
:103DB0003031323334353637383941424344454661
:103DC0000000000000400000004000000040000033
:103DD000004000000000010000000200000002009E
:103DE00000000200000002000000020000000200CB
:103DF0000000020000400000004000000040000001
:103E0000004000000000010000000200000002006D
:103E1000000002000000020000000200000002009A
:103E200000000200000000000D1B0008ED1D00084E
:103E3000991E000840004000303700203037002035
:103E40000100000040370020800000004001000019
:103E5000050000006D61696E00000000743E0008FE
:103E6000483700204039002001000000713500086B
:103E70000000000069646C65000000000000802AFA
:103E800000020000AAAAAAAA00000000FFFF00008A
:103E90000000000000A00A00040040000000000034
:103EA000AAAAAAAA00000000FFFF0000000000006C
:103EB000000000001000004000000000AAAAAAAA0A
:103EC00010000040FFFF00000000000000000000A4
:103ED00080699A0100000000AAAAAAAA40555501CB
:103EE000FFFF0000007070077770000000000040C6
:103EF00000000000AAAAAAAA00000040FFFF0000DC
:103F000000000000000000000000000000000000B1
:103F1000AAAAAAAA00000000FFFF000000000000FB
:103F2000000000000000000000000000AAAAAAAAE9
:103F300000000000FFFF0000000000000000000083
:103F40000004000000000000AAAA00000004000015
:103F5000FF00000000000000000000000000000062
:103F600000000000AAAAAA0000000000FF0F000045
:103F70000000000000000000000000000000000041
:103F80000000000000000000000000000000000031
:103F90000000000000000000000000000000000021
:103FA0000000000000000000000000000000000011
:103FB000FF0096000000000804000000983D000883
:103FC00000000000000000000000000000000000F1
:083FD0000000000000000000E9
:00000001FF
